:100000000C946C010C9494010C9494010C94940144
:100010000C9494010C9494010C9494010C9494010C
:100020000C9494010C9494010C94681A0C943A1B4F
:100030000C948D150C9494010C9494010C949401DF
:100040000C9494010C9494010C9494010C949401DC
:100050000C9494010C9415160C9494010C94940136
:100060000C9494010C9494010C9494010C949401BC
:100070000C9494010C9494010C9494010C949401AC
:100080000C9494010C9494010C9494010C9494019C
:100090000C9494010C9494010C9494010C9494018C
:1000A0000C9494010C9494010C949401030603069F
:1000B0002F062F069706C207C207C207B5064E07CE
:1000C0005F075F07A71BCE1BC61CCE1BC61C1A1CD6
:1000D0003D1CC61C941CA31C04001600070009004C
:1000E0000B000A001D001B0006001900000005009F
:1000F00014001A00080015001C0017001E001F0045
:1001000020002100230022002E00260024002D00C4
:10011000250027003000120018002F000C001300EB
:1001200028000F000D0034000E00330031003600AF
:1001300038001100100037002B002C0035002A0079
:1001400000002900E000E300E1008200E20050002E
:100150004F005100520000000000630000005500F5
:100160000000570000005300000000000000540091
:10017000580000005600000000002E0062005900E8
:100180005A005B005C005D005E005F0000006000E4
:1001900061000000000000003E003F0040003C0005
:1001A00041004200000044000000460000004700FB
:1001B00000004300000045000000480049004A00DC
:1001C0004B004C003D004D003B004E003A00E50066
:1001D000E600E4000000B0002E03410044004200AD
:1001E00020006B006500790062006F006100720002
:1001F0006400200063006F006E00760065007200EE
:100200007400650072000000080351004D004B00AF
:1002100000000403090409023B00020100A0FA09DE
:100220000400000103010100092111010001224025
:100230000007058103080001090401000103000013
:10024000000921110100012232000705820320006C
:10025000011201000200000008EDFEDB0A010101AD
:1002600002000105010980A101850319012AB700D7
:10027000150126B700950175108100C0050C090114
:10028000A101850419012AA002150126A0029501E9
:1002900075108100C005010906A101050719E029B3
:1002A000E715002501950875018102950175088102
:1002B000010507190029FF150026FF00950675089E
:1002C000810005081901290595057501910295011F
:1002D00075039101C000801411241FBECFEFDAE036
:1002E000DEBFCDBF11E0A0E0B1E0E2EAFAE302C078
:1002F00005900D92A838B107D9F722E0A8E8B1E03F
:1003000001C01D92A539B207E1F711E0CCE6D1E0BA
:1003100004C02197FE010E94FA1CCB36D107C9F711
:100320000E9428120C944F1D0C940000282F277057
:10033000E82FE695E695E695EF70F0E0E457FE4F7E
:1003400087FF0AC081E090E001C0880F2A95EAF794
:1003500080959081892308C081E090E001C0880FDA
:100360002A95EAF79081892B8083089508950C944B
:10037000B6010C94B7010C94B6010E9482022FEFD3
:1003800087EA91E6215080409040E1F700C00000EC
:10039000ECE8F1E0119221E0EC39F207D9F70C9486
:1003A000C8031F93CF93DF93C0910001D091010147
:1003B0008FEF9FEF9093010180930001CF3F8FEF6C
:1003C000D80799F480918A0190918B010E940616BA
:1003D0000C9710F480E02EC00E94EE1590938B01D4
:1003E00080938A010E941D03EC01209799F3CF3777
:1003F0008FE7D80711F48FE705C0CF3F8FEFD807FD
:1004000021F48FEF0E94960112C0DF3F21F40E9479
:10041000BD018C2F0FC08D2F0E949601CF3F39F068
:10042000DC2FCC27CF6FD0930101C09300010E9435
:10043000CA0381E0DF91CF911F9108950895E82FBD
:10044000F0E0E457FE4F80810895509A83E091E0F8
:100450000197F1F700C0000050989AEB9A95F1F7D8
:1004600000C00895509A8AEB8A95F1F700C0509821
:1004700083E091E00197F1F700C000000895EF924A
:10048000FF920F931F93CF93DF93C0E0D0E090E8EB
:10049000E92EF12C082F10E0C7010C2E02C0959513
:1004A00087950A94E2F780239123892B19F00E9403
:1004B000320202C00E9425022196C830D10561F7A0
:1004C000DF91CF911F910F91FF90EF900895509A77
:1004D00083EF9BE00197F1F700C000000C9432021B
:1004E000489B06C023E02A95F1F700000197C1F769
:1004F0000895489906C023E02A95F1F70000019776
:10050000C1F70895589850980895EF92FF920F936D
:100510001F93CF93DF93C82F162F7A01D22F80E03D
:10052000422F50E0282F082E000C330B24173507DC
:1005300034F4F701E20FF31F10828F5FF3CFF894CA
:100540000E94670280E1C89F90011124812F8C6076
:10055000822B0E943F020E94250284EF91E00E94BC
:100560007902892B91F084EF91E00E947002892B2F
:1005700061F088E290E00E947902892B31F084E6F4
:1005800090E00E947002892B19F4789480E02BC0CF
:10059000C0E082E890E00E9479028823F9F08C01A3
:1005A0001127C8010E9470028823C1F09C2F9695E4
:1005B000969596959D1780F4F701E90FF11D9081AE
:1005C000990F22E830E0201B310B081B110920177E
:1005D00031070CF491609083CF5FD9F678948C2F1B
:1005E000869586958695DF91CF911F910F91FF900B
:1005F000EF900895CF93DF93CDB7DEB728970FB66E
:10060000F894DEBF0FBECDBF28E0AE014F5F5F4F55
:100610000E948502823031F489819A819827892746
:10062000982702C080E090E028960FB6F894DEBFCD
:100630000FBECDBFDF91CF91089560E082E00C94B2
:10064000FA02EF92FF921F93CF93DF93D82F162FCA
:100650007A01C22FF8940E94670280E1D89F90012E
:100660001124812F8860822B0E943F020E94250264
:100670008FE193E00197F1F700C000000E94320281
:1006800010E0D0E0812F012E000C990B8C179D07F4
:1006900044F4F701E80FF91F80810E943F021F5FB9
:1006A000F1CF0E9425027894DF91CF911F91FF90A6
:1006B000EF900895CF93DF9300D0CDB7DEB7498395
:1006C0002A8322E0AE014F5F5F4F0E9421030F900B
:1006D0000F90DF91CF910895282F277040E062E0BE
:1006E00082E00C945A0380950C946C0381E0089589
:1006F00081E008950C94780308950C947C031F9373
:10070000CF93DF9300D000D01F92CDB7DEB74983DF
:100710005A836B8330919D0189819A81311114C074
:10072000662359F0222349F00E94FB09182F682FF5
:1007300089819A810E94A40903C00E94CF09182FC1
:1007400069817A81812F04C00E94FB0969817A81C5
:100750000F900F900F900F900F90DF91CF911F91FE
:100760000C940411FC01262F408151816281738118
:1007700084810C947F0381E00895CF93DF93EC0193
:1007800060E00E94B203BE01DF91CF910C947D0323
:100790000C94B9010C94BB0108950E944E080E946C
:1007A000CC032FEF84E39CE0215080409040E1F7A0
:1007B00000C000000C943B160F931F93CF93DF9360
:1007C0008C0161E00E94B203EC01B8010E947A033F
:1007D0008823F1F1B801CE010E9421148823C1F1D0
:1007E000B801CE010E943512882391F1B801CE01E3
:1007F0000E947D13882361F1F8018281882309F129
:10080000CB358DE5D807C1F050F4C115FCE5DF0705
:1008100081F0CF3DDC45A9F40E942C0F19C0CC35E6
:10082000EDE5DE0761F0CD35DD4559F40E94750E2A
:1008300008C00E94CD030CC00E947E0E02C00E9420
:10084000810EC801DF91CF911F910F910C94760317
:1008500080E0DF91CF911F910F9108950E94701554
:100860000C9437040E943A040C947615089580E0A5
:100870000C9473030E94C3140C9473030E94C3145A
:1008800090919C01891721F080939C010C94730333
:100890000895CF93DF93CDB7DEB72B970FB6F894BB
:1008A000DEBF0FBECDBF4F83588769877A878B879E
:1008B00061110E94C10D9E012F5F3F4F86E0F9013B
:1008C00011928A95E9F785E0FE013796D9010190EA
:1008D0000D928A95E1F789819A814C815D81452B42
:1008E00031F09F3F31F491E08F3F19F403C091E064
:1008F00001C090E090FF09C049815A816B817C81E1
:100900008D819E810E94E20C05C0C9010E94BB033B
:100910008111F2CF2B960FB6F894DEBF0FBECDBF7C
:10092000DF91CF910895FC01808191810E943D0A61
:100930000895CF93882309F49CC0C82F8238C1F44E
:100940000E94C31481FD95C069E3809104019091D8
:1009500005010E9448150E94E30D2FEF81EE94E0FF
:10096000215080409040E1F700C0000069E319C0C9
:10097000833801F50E94C31480FD7BC063E580913C
:100980000401909105010E9448150E94E30D2FEF8C
:1009900081EE94E0215080409040E1F700C00000DB
:1009A00063E580910401909105010E944A15CF9161
:1009B0000C94E30D8438C1F40E94C31482FD59C025
:1009C00067E480910401909105010E9448150E94FE
:1009D000E30D2FEF81EE94E0215080409040E1F74D
:1009E00000C0000067E4DDCF8CEF8C0F813AD0F4BB
:1009F0006C2F80910401909105010E9412158823AB
:100A000049F06C2F80910401909105010E944A15D4
:100A10000E94E30D6C2F80910401909105010E94CA
:100A20004815C5CF80E28C0F883048F4C77081E04C
:100A300001C0880FCA95EAF70E94A40DB8CFEBE574
:100A4000EC0FE33040F4F0E0EF5BFE4F808190E08C
:100A5000CF910C94DA14C85AC73158F4EC2FF0E057
:100A6000EE0FFF1FED5EFE4F80819181CF910C94C0
:100A7000F014CF910895882309F45BC0682F823861
:100A800079F40E94C31481FF54C069E3809104018A
:100A9000909105010E9448150E94E30D69E310C082
:100AA0008338B1F40E94C31480FF43C063E5809192
:100AB0000401909105010E9448150E94E30D63E531
:100AC00080910401909105010E944A150C94E30D58
:100AD000843879F40E94C31482FF2BC067E48091AC
:100AE0000401909105010E9448150E94E30D67E4FE
:100AF000E7CF8CEF860F813A18F380E2860F8830BB
:100B000048F4677081E001C0880F6A95EAF70E9497
:100B1000AA0DDCCF8BE5860F833020F480E090E0D7
:100B20000C94DA14685A673120F480E090E00C9459
:100B3000F01408951F93CF93DF93182FEB010E94B9
:100B40009904209741F08FE99FE00197F1F700C0E9
:100B500000002197F6CF812FDF91CF911F910C9448
:100B60003B05893319F060E070E002C060E570E099
:100B70000C949A05882321F00E94A40D0C94E30D97
:100B80000895882321F00E94AA0D0C94E30D089586
:100B9000CF92DF92EF92FF920F931F93CF93DF9349
:100BA0007C01D62FC72FFC011281058102950F70A1
:100BB0000E949A0D8823B9F01123A9F08C2F807F11
:100BC000803421F080E28D0F883068F080918302BC
:100BD00082FD09C082E00E94430E0E949A0D91E0BE
:100BE000D82ED92601C0D12CCC2EC2948FE0C82299
:100BF0008C2D90E08C30910508F0C4C1FC01EA5ABC
:100C0000FF4F0C94FA1C8C2F807FCF70882311F03B
:100C1000C295C07F112399F0CC2309F49FC180E2D3
:100C20008D0F883010F0D11104C08C2F0E94A40DBC
:100C300003C08C2F0E94B40D0E94E30D8FC18D2F35
:100C40000E943B05CC2309F49DC180E28D0F8830C2
:100C500038F1DD2329F18C2F0E94BA0D24C08C2F8E
:100C6000807FCF70803211F0C295C07FDD2319F0F4
:100C7000D130A1F13DC08091830282FF17C01123C2
:100C800049F0CC2329F08C2F0E94A40D0E94E30D83
:100C900080E065C180E00E943B05CC2309F472C16D
:100CA0008C2F0E94AA0D0E94E30D6CC1112371F0DC
:100CB000002341F0013031F40E94C40D8C2B0E94BE
:100CC000CC0D60C10E94C40D8C2B1DC0002319F0F7
:100CD000013009F457C10E94D90D25C0112321F01C
:100CE000063008F04FC10EC0053008F04BC11BC0E4
:100CF000112361F0002331F0F701858180FF2EC1BF
:100D00008F7085838C2F0E94BA053CC1002359F057
:100D1000D93309F034C1FFEF07EE13E0F150004082
:100D20001040E1F72AC18C2F0E94C1052BC18C2FE6
:100D300086958695837019F0813061F023C1112367
:100D400021F08D2F9C2F937002C080E090E00E94D4
:100D5000DA1420C1112321F08D2F9C2F937002C033
:100D600080E090E00E94F01415C18C2F837009F090
:100D700047C011110BC12D2F229526952770220FE8
:100D8000220F6D2F6F70862F90E0A0E0B0E0022E52
:100D900004C0880F991FAA1FBB1F0A94D2F7D4FF63
:100DA00010C04FE050E060E070E004C0440F551FF9
:100DB000661F771F2A95D2F74095509560957095DC
:100DC00003C040E050E0BA01C695C695C3708A01E1
:100DD0009B01082B192B2A2B3B2BC901B801C230D0
:100DE00049F058F4C13019F00E94BA08CFC00E94EF
:100DF000A808CCC00E94CC08C9C00E94A608C6C0E2
:100E0000112319F08C2F817001C08695882309F475
:100E1000BDC02D2F229526952770220F220F6D2FF2
:100E20006F70862F90E0A0E0B0E0022E04C0880F23
:100E3000991FAA1FBB1F0A94D2F7D4FF10C04FE01E
:100E400050E060E070E004C0440F551F661F771F3C
:100E50002A95D2F7409550956095709503C040E073
:100E600050E0BA01C695C695C3708A019B01082B54
:100E7000192B2A2B3B2BC901B801C23049F058F479
:100E8000C13019F00E947F0981C00E946D097EC0A7
:100E90000E9491097BC00E94E00878C0CF701123A6
:100EA00039F08C2F0E9406098D2F0E94BA056EC062
:100EB0008D2F0E94C1058C2F0E94270967C0D23F49
:100EC00021F128F4D03F41F0D13FC1F043C0D33FDE
:100ED00019F1D43F79F03EC0112341F0053008F0FC
:100EE00051C08C2F8F710E944C094CC0063008F005
:100EF00049C0F7CF8091830282FF18C0112339F0D7
:100F00008C2F8F710E9406093DC01123C9F38C2FCD
:100F10008F710E94270936C0112329F08C2F8F7101
:100F20000E94F1082FC00E94EC082CC0112349F048
:100F3000CF718C2F0E94060963E08C2F0E94280E2F
:100F400021C081E00E94430E0230E0F082E00E9466
:100F5000430E18C0112331F0002391F28D2F0E940F
:100F6000990410C0002399F2D93349F41FEF27EEFA
:100F700033E0115020403040E1F700C000008D2FD9
:100F80000E943B0588EF8C0D843020F40E94C3142E
:100F90000E947303DD20C9F00E94960D80FD15C0EC
:100FA000F70112820E94900D0E940609C7010E945B
:100FB00006080E94900DDF91CF911F910F91FF9035
:100FC000EF90DF90CF900C942709DF91CF911F9184
:100FD0000F91FF90EF90DF90CF9008950F931F93A4
:100FE000CF93DF93EC01688179818A810E94480A5E
:100FF0008C010E94A3090E949408B801CE010E94AE
:10100000C805DF91CF911F910F910895CF93DF9382
:10101000EC01988189812B813C81232B31F08F3F1A
:1010200031F481E09F3F19F403C081E001C080E00A
:1010300080FD1DC0CE010E94DC03811110C00E9402
:101040009A0D8823A1F08A81882389F080918302F8
:1010500082FD0DC082E0DF91CF910C94430ECE0152
:101060000E94EE07CE01DF91CF910C94BD03DF917A
:10107000CF91089580E090E00E94DA1480E090E043
:101080000E94F0140E94C10D0C94E30D80910401A4
:10109000909105010E944C150C943A080E94B10DE4
:1010A0000C94460892959F70963079F010F4925007
:1010B00001C09A50923068F4803F69F018F4883E7D
:1010C00040F409C0843F29F406C0883E20F0813FE7
:1010D00011F080E0089581E00895FC018081918104
:1010E0000E943D0A0E9452080895CF93DF9300D0DA
:1010F00000D01F92CDB7DEB70F900F900F900F90DA
:101100000F90DF91CF910895CF93DF9300D000D05F
:1011100000D0CDB7DEB726960FB6F894DEBF0FBE6F
:10112000CDBFDF91CF910895089508950C9495084F
:101130000C9496080E9498086093F2017093F30152
:101140008093F4019093F5010C943A080C949A085A
:101150000F931F930091F2011091F3012091F4017C
:101160003091F501602B712B822B932B1F910F91E6
:101170000C949A080F931F930091F2011091F301C0
:101180002091F4013091F501602371238223932390
:101190001F910F910C949A080F931F930091F201E5
:1011A0001091F3012091F4013091F501602771272E
:1011B000822793271F910F910C949A080C949508FD
:1011C0000E94DE086093EE017093EF018093F001BE
:1011D0009093F1010C943A0860E070E0CB010C941C
:1011E000E0080F931F9341E050E060E070E08A0157
:1011F0009B0104C0000F111F221F331F8A95D2F7D5
:10120000C901B8011F910F910C94E0080F931F932F
:1012100041E050E060E070E004C0440F551F661FDD
:10122000771F8A95D2F78091EE019091EF01A091FE
:10123000F001B091F1018A019B01082B192B2A2B97
:101240003B2BC901B8011F910F910C94E0080F933B
:101250001F9341E050E060E070E004C0440F551F70
:10126000661F771F8A95D2F74095509560957095C7
:101270008091EE019091EF01A091F001B091F10108
:101280008A019B01082319232A233B23C901B801A2
:101290001F910F910C94E0080F931F9341E050E0D1
:1012A00060E070E004C0440F551F661F771F8A95E9
:1012B000D2F78091EE019091EF01A091F001B091F1
:1012C000F1018A019B01082719272A273B27C90119
:1012D000B8011F910F910C94E0080F931F93009198
:1012E000EE011091EF012091F0013091F101602B9E
:1012F000712B822B932B1F910F910C94E0080F936D
:101300001F930091EE011091EF012091F0013091B7
:10131000F10160237123822393231F910F910C9479
:10132000E0080F931F930091EE011091EF012091BF
:10133000F0013091F10160277127822793271F91D7
:101340000F910C94E008089528E0929F800D1124DD
:10135000E82FE695E695E695877051E001C0550FB8
:101360008A95EAF785E0E89FF0011124E256FE4FE6
:1013700020E030E070E04081CB01022E02C0969563
:1013800087950A94E2F781708195842785238427C5
:1013900081932F5F3F4F2530310569F7089528E08D
:1013A000929F800D1124682F669566956695982FFB
:1013B000977085E0689FB001112440E050E080E024
:1013C000FB01E40FF51FE256FE4F208130E0092EAD
:1013D00002C0369527950A94E2F721703327042E30
:1013E00001C0220F0A94EAF7822B4F5F5F4F45300E
:1013F000510531F70895BF92CF92DF92EF92FF929D
:101400000F931F93CF93DF938C01C090EE01D09088
:10141000EF01E090F001F090F1018091F2019091E4
:10142000F301A091F401B091F501C82AD92AEA2A62
:10143000FB2ACFE1D0E0D701C6010C2E04C0B6953F
:10144000A795979587950A94D2F780FD04C02197B8
:1014500090F7B12C07C0BC2EB8018C2F0E94191137
:101460000197A9F38B2DDF91CF911F910F91FF90E1
:10147000EF90DF90CF90BF900895CF93DF93EC0172
:101480000E94FB09BE010E941911DF91CF910895BE
:101490001F93CF93DF93EB0190919D01992321F04E
:1014A000CB010E943D0A13C0882349F0CB010E9462
:1014B000FB09182F682FCE010E94A40904C0CB019C
:1014C0000E94CF09182FBE01812F0E941911DF91B0
:1014D000CF911F9108951F93CF93DF93C091F60191
:1014E00016E08091F701C81799F0D0E01C9FF00139
:1014F0001D9FF00D1124E850FE4F40815181628103
:101500007381848195810E9484082196C770E9CFF8
:10151000DF91CF911F9108954091280250912902A7
:1015200060912A0270912B0280912C0290912D02E1
:101530000C948408EF92FF920F931F93CF93DF9345
:1015400080912D0282958F7009F065C080912A02EA
:10155000882309F460C08091F601F090F7011091A2
:1015600028020091290260912B0270912C0291E0D7
:101570001F3F09F090E0C0910201D0910301292F93
:1015800096E0E92E8F1509F446C06115710521F02A
:101590000F3F21F030E003C031E001C0322F90E076
:1015A00030FD36C0E89EF001E99EF00D1124DF0108
:1015B000A850BE4F11963C911197301329C03C9111
:1015C000311326C012963C911297311121C0139607
:1015D0004D915C911497461B570B4C175D07C0F457
:1015E00080912D028F70806180932D02E350FE4F19
:1015F00080818F708061808388E292E00E9406087B
:10160000DF91CF911F910F91FF90EF900C946B0A97
:1016100001968770B7CFDF91CF911F910F91FF9007
:10162000EF9008959F92AF92BF92CF92DF92EF9288
:10163000FF920F931F93CF93DF93CDB7DEB76197E0
:101640000FB6F894DEBF0FBECDBF8C0185E0F80168
:10165000DE011D9601900D928A95E1F7D801129650
:10166000EC9090912802E091290220912B02309178
:101670002C022115310531F0EF3F31F481E09F3F1D
:1016800019F403C081E001C080E0B82FB1709B2E37
:1016900080FD47C1D8014C9111965C91119713962A
:1016A000AD90BC90149788E2C82E82E0D82EF090BE
:1016B0002A02B501621B730B2091020130910301D4
:1016C000FF2009F4D9C080912D026217730708F03A
:1016D00095C0282F207F09F052C05E1313C0491314
:1016E00011C0FE2CE1100EC08F70806180932D021E
:1016F0000E948C0AC6010E94060880912D02F80102
:1017000085834DC1AB2831F05F3F31F481E04F3F1D
:1017100019F403C081E001C080E080FD03C081E0D6
:101720008E2502C080E090E0F82FF170FF2E80FF40
:101730001CC08091F6012091F70136E0821709F470
:101740000BC190E0389FF001399FF00D1124E85053
:10175000FE4F6181561306C06081461303C062814B
:10176000E61203C001968770E9CFFE2CEE2009F443
:1017700016C180912D02816080932D0254C05E13AA
:1017800006C0491304C0E11002C0F80199C0C801A5
:101790000E946D08882361F1EE2051F120912D0205
:1017A000822F82958F7090E0029774F080912802CA
:1017B0009091290298878F831986BB86AA862C87E9
:1017C000CE0107960E94060886E0F801A8E2B2E082
:1017D00001900D928A95E1F70E949A0A0E948C0A64
:1017E0000AC05E1711F1C8010E946D0881112CC05A
:1017F000C8010E940608FF24F394D1C0282F207F3F
:1018000081F77A2DB98AA88A6E2D89890E94750878
:1018100088E292E00E94060886E0D6011D928A9531
:10182000E9F70E948C0AF12CBAC04913DCCFE11011
:10183000DACFF8018583C8010E94060886E0D60148
:101840001D928A95E9F7ABC0EE2091F220912D020E
:10185000822F82958F7090E002970CF4B5CF809123
:101860002802909129029A8389831B82BD82AC82CF
:101870002E83CE010196A6CF6217730708F044C0ED
:10188000FE2CEE2009F4B4CF5E1330C049132EC0F5
:1018900020912D0220FD21C0822F82958F70482F2C
:1018A00050E041155105C9F0F80125834F3051052D
:1018B00041F08F5F982F9295907F822F8F70892BA8
:1018C0008583C8010E94060886E0F801A8E2B2E01C
:1018D00001900D928A95E1F73CC086E0F801A8E2FC
:1018E000B2E001900D928A95E1F759C0C8010E94BB
:1018F0006D08811169CF80912D02816080932D0246
:10190000C8010E9406084BC07A2DB98AA88A6E2D9C
:1019100089890E94750886E0D6011D928A95E9F7AB
:1019200018C0EE2009F464CFC8010E946D08F82E9B
:10193000882309F45DCF86E0F801A8E2B2E00190C7
:101940000D928A95E1F788E292E00E9493040E944A
:101950009A0A0E948C0A23C04D875E878D859E85DA
:101960000E943D0A292F22952F70223028F49F7063
:1019700039F0811105C00BC0243028F49F7049F460
:10198000805E883020F0C8010E9406089F2CF92C48
:1019900006C0D80115969C91907F91F7F8CF8F2DB6
:1019A00061960FB6F894DEBF0FBECDBFDF91CF9129
:1019B0001F910F91FF90EF90DF90CF90BF90AF906D
:1019C0009F9008951F93CF93DF93CDB7DEB72C97E9
:1019D0000FB6F894DEBF0FBECDBF4F83588769871F
:1019E0007A878B879C87CE0107960E94120B8823EB
:1019F000D1F09F8188852A853B85232B31F08F3F4D
:101A000031F481E09F3F19F403C081E001C080E020
:101A100080FD47C04F81588569857A858B859C8577
:101A20000E9484083EC086E0FE013796DE011196D2
:101A300001900D928A95E1F7FF81E8856A857B85A3
:101A40006115710531F0EF3F31F481E0FF3F19F48A
:101A500003C081E001C080E080FD23C02091F70138
:101A600030E0C9010196877099274091F60150E056
:101A700084179507F1F1F983EA837D836C8396E0FF
:101A8000929FD001939FB00D1124A850BE4FFE012C
:101A9000319601900D929A95E1F78093F7010E949B
:101AA0006B0A16E08091F6019091F701891771F1A8
:101AB000189FC001112488509E4F0E94120B88234A
:101AC00029F1E091F6011E9FF0011124E850FE4F2C
:101AD0004081518162817381848195810E94840853
:101AE0008091F60190E00196877099278093F60126
:101AF000D9CF0E944E081092F7011092F601E8E249
:101B0000F2E086E0DF011D928A95E9F72C960FB688
:101B1000F894DEBF0FBECDBFDF91CF911F91089526
:101B20008091360285958595859508958091360238
:101B30008770089590913602977081E009F480E0F3
:101B4000089580914102089590914102892B8093DC
:101B5000410208958095909141028923809341022A
:101B6000089510924102089590914002892B80932C
:101B7000400208958095909140028923809340020D
:101B800008951092400208958091370208950895B3
:101B90000C94C70D0C94C80D9091830292FD08C05F
:101BA00090913702981721F0809337020C94CA0D58
:101BB000089580913702882329F01092370280E03F
:101BC0000C94CA0D0895CF93DF93E0910401F09136
:101BD0000501809141028083E0910401F0910501AB
:101BE000908180914002892B8083809137028823E5
:101BF00081F0E0910401F09105019081892B8083AF
:101C000080910401909105010E94061581110E94A6
:101C1000D90DC0910401D091050148E050E06EE279
:101C200072E0CE010E94001D892B69F088E0FE0160
:101C3000AEE2B2E001900D928A95E1F7CE01DF911C
:101C4000CF910C94CF14DF91CF9108950C94C70DD0
:101C50009091830292FD10C098E0899F9001112419
:101C6000262B209336020E94060980913602859524
:101C7000859585950C94260E0C94060910923602D3
:101C800080E00C94260E209136028095822380936A
:101C90003602982F977099F430E0482F082E000CE8
:101CA000550B2417350759F09091830292FD07C018
:101CB0008595859585950E9427090C943E0E08957B
:101CC0009091830292FB222720F9281769F080FB6C
:101CD00092F99093830280918202909183020E94F4
:101CE000A80E82E00C94430E08958091830282FB3B
:101CF000882780F991E089270C94600E81E00C948C
:101D0000600E80E00C94600E80E090E00E94151D53
:101D100021E0893E9E4F09F020E0822F089582E065
:101D200090E00C940D1D83E090E00C940D1DCF937A
:101D300084E090E00E940D1DC82F82E290E00E9496
:101D40000D1D2C2F30E0A901582BCA01CF91089509
:101D5000CF93C92F682F84E090E00E941B1D6C2F49
:101D600082E290E0CF910C941B1DAB01BC018FE08F
:101D700090E00C942D1DAB01BC0183E190E00C942C
:101D80002D1D60E070E0CB010C94BB0E60E070E0B4
:101D9000CB010E94B50E0C94C10E69EE7EEF80E07F
:101DA00090E00E94391D60E082E090E00E941B1DDF
:101DB00060E083E090E00E941B1D1092F2011092FF
:101DC000F3011092F4011092F50160E084E090E0DC
:101DD0000E941B1D60E082E290E00E941B1D60E0FB
:101DE00085E090E00E941B1D60E086E090E00E948C
:101DF0001B1D6FEF87E090E00E941B1D40E050E04C
:101E0000BA0188E090E00E942D1D60E08DE090E036
:101E10000E941B1D40E050E0BA0188E190E00E9462
:101E20002D1D60E087E190E00E941B1D40E050E026
:101E3000BA018CE190E00E942D1D60E070E080E22C
:101E400090E00E94391D40E050E0BA0188E190E046
:101E50000E942D1D0C94C60E0C94CD0E682F8EE0A2
:101E600090E00C941B1D0E94FA156093560270932B
:101E700057028093580290935902609352027093D4
:101E800053028093540290935502089585B7806859
:101E900085BF85B7806885BF089581E008950C945B
:101EA0004D0F08950C94510F0C94510F0C94540F36
:101EB0000C94510F0C94580F0C94510F0E94460F24
:101EC00085EF91E10E94B9140E945C0F0C945A0FA7
:101ED0000E94520F0C94510F0E94F8110C9436047A
:101EE0000E94E5150E94BD010E946C0F0C94560FD4
:101EF0008F929F92AF92BF92CF92DF92EF92FF921A
:101F00000F931F93CF93DF93CDB7DEB72A970FB60A
:101F1000F894DEBF0FBECDBF0E94D101982E811173
:101F20000E94330F82E4A82E82E0B82E00E010E079
:101F3000802E802F0E941F02D82EF501C1905F01D4
:101F4000C826B1F40F5F1F4F0031110589F78FEFDD
:101F500089838A831B820E94EE158160782F9D837E
:101F60008C8349815A816B818D810E9449042FC0E5
:101F700080915A0281FD0E941E02E12CFF24F394FD
:101F80008C2D8F21F1F00E944F0F882399F0EE8263
:101F90008F82DF2081E009F480E088870E94EE15BF
:101FA0008160782F9A8789874E815F8168858A85CD
:101FB0000E944904F801EE5BFD4F8081F826F08213
:101FC00006C0E394FF0CF8E0EF12DACFBBCF81E05C
:101FD000911001C080E02A960FB6F894DEBF0FBEC4
:101FE000CDBFDF91CF911F910F91FF90EF90DF90C8
:101FF000CF90BF90AF909F908F9008950E94780FE0
:102000000C943E04CF93DF930E941E11EC018115C6
:1020100022E59207E8F5811531E5930708F0B6C08F
:10202000883E910528F5803E910508F0E9C0883A80
:10203000910570F4853A910508F07AC081309105D8
:1020400009F473C008F4D9C0049708F0D9C0D5C00A
:102050008F3B910508F0D1C0C85AD0E0CC0FDD1FEE
:10206000CC5BDE4F0990D881C02DCE019464C9C0ED
:10207000811540E5940708F069C0811550E4950783
:1020800008F060C09A9581159F4108F4B9C0B5C0A9
:10209000811536E5930728F5811545E5940708F085
:1020A00092C0811554E5950708F087C0AC014370D4
:1020B0005527282F26952695C115D34508F06CC0C5
:1020C00081E090E002C0880F991F4A95E2F740E254
:1020D000249F90011124EC01C22BD32BCE019C68CC
:1020E00090C081152AE5920780F4811539E59307A0
:1020F00008F072C0811548E5940708F47EC0D82F17
:10210000CC27CE01806F906A7CC09056811590429A
:1021100008F073C08D2F8F710E94B211DD27D0623D
:102120008F71AE01582BCA016CC081E090E069C08C
:10213000C55AD0E0CE58DE4F8881C82FD0E0CE01FE
:1021400090645FC0DF70CE01906A5BC074E09695CA
:1021500087957A95E1F7282F23703C2F337081E023
:1021600090E002C0880F991F3A95E2F79C68AC0195
:10217000522B9A019C2F9F709695969550E2959FB1
:10218000E0011124C9018C2B9D2B3BC0D82FCC27FB
:10219000CE01816F906A35C081E090E002C0880F67
:1021A000991F4A95E2F750E2259F90011124EC0116
:1021B000C22BD32BCE019A6824C0D82FCC27CE01B6
:1021C000846F906A1EC00E94B2118F7190E0D82F68
:1021D000CC27CE01906215C08F700E94B21194E09E
:1021E000D695C7959A95E1F7CF70D0E0DC2FCC2734
:1021F000D0699E01282BC90104C080E090E001C095
:10220000CE01DF91CF910895E72FF0E090E1899F13
:10221000E00DF11D112483E0EE0FFF1F8A95E1F719
:10222000E60FF11DEE0FFF1FE852FF4F85919491CD
:1022300008950E9404110E940210089582389105A9
:1022400069F1B0F48133910509F46DC048F4893225
:10225000910509F463C08A32910509F469C00895B3
:102260008533910509F455C089339105B9F0089576
:10227000833E910569F138F4803E9105B1F0823ECC
:10228000910509F10895863E9105A9F1873E9105D2
:10229000B9F1843E910509F064C023C02091820207
:1022A00020FD4FC021FD4DC008958091820280FD28
:1022B00044C08091830280FF44C08091820284FDEB
:1022C00042C083EE4DC08091820282FF38C0F5CFBC
:1022D0008091820282FD33C08091830280FD31C0F3
:1022E000ECCF8091830281FF32C08091820284FD15
:1022F0002AC087EE35C08091820283FF26C0F5CFC9
:102300008091820283FD21C08091830281FD1FC0E4
:10231000ECCF8091820285FD1CC01DC0809182029D
:1023200085FD19C016C08091820286FD16C017C0B7
:102330008091820286FD13C010C089E311C082EE35
:102340000FC080EE0DC080E00BC086EE09C084EEA9
:1023500007C089E205C085E303C08AE201C081E3CA
:1023600090E008959091820292FF0DC0282F28716D
:10237000283019F4877F846006C0282F2471243008
:1023800011F48B7F886093FF0DC0282F28712831AE
:1023900019F4877E846106C0282F2471243111F43A
:1023A0008B7E88612091830220FF0DC0382F387109
:1023B000383019F4877F816006C0382F3171313091
:1023C00011F48E7F886021FF0DC0282F28712831DD
:1023D00019F4877E816106C0282F2171213111F403
:1023E0008E7E886194FD877E089580E0089508952B
:1023F0000E94840E811102C00E942C0F0E948F0E39
:1024000080935A020E94970E9093830280938202D7
:102410000E94F7110E94930E682F70E080E090E018
:102420000E94A6086091EE017091EF018091F00189
:102430009091F1010C94DE080E94C0170E94700F69
:102440000C94CC170E94D0170E94FE0F0C94EA1730
:102450000E948C150E94A7170E945E0F0E941C12FA
:102460000E9422120E94680FFBCFCF93DF93EC01F2
:10247000FB018281882309F43CC1C430FDE5DF07FC
:1024800060F4CB3F9CE5D90788F49E0122503C457F
:102490002431310508F02EC109C0C236EDE5DE0752
:1024A00029F0C63AFDE5DF0709F024C10E94970E26
:1024B0009093830280938202C1318CE5D80709F49E
:1024C000C6C008F042C0C930ECE5DE0709F49BC085
:1024D00000F5C5308CE5D80709F485C078F4C33021
:1024E000ECE5DE0709F478C008F07AC0C230DC45BC
:1024F00009F0F5C0809182028160EFC0C7309CE591
:10250000D90709F478C008F07AC08091820280610E
:10251000E4C0CD30FCE5DF0709F487C058F4CB30C8
:102520009CE5D90709F479C008F07BC0809182024C
:1025300088606FC0CF30FCE5DF0709F480C008F089
:1025400082C080918202877FC8C0CE3F9CE5D907B8
:1025500009F471C000F5C531FCE5DF0709F485C059
:1025600068F4C3319CE5D90709F475C008F095C03B
:102570000E944E08809182028F77AFC0CC3FFCE56D
:10258000DF07A9F108F054C0CB3FDC4509F0A7C034
:102590008091830240C0C230EDE5DE0709F489C0B6
:1025A00058F4C1158DE5D80709F45AC008F069C080
:1025B0008091830282602FC0C236EDE5DE0709F408
:1025C0007CC0C63AFDE5DF0709F481C0C330DD45B4
:1025D00009F085C080E06EC08091820282607DC07B
:1025E0008091820216C080918202886076C08091BC
:1025F000830282604FC08091820280626EC08091AF
:10260000820280646AC00E944E08809182028068C3
:1026100064C0846062C081603DC0809182028E7F10
:102620005CC0809182028D7F58C08091820216C06A
:102630008091830218C0809183028D7F2BC080918E
:1026400082028F7E4AC0809182028F7D46C0809137
:1026500082028F7B42C080918202877F8B7F3DC048
:10266000809183028D7F8E7F15C08091820282FBD4
:10267000222720F991E0922790FB82F990FB83F9C1
:102680002CC080918302982F909591708E7F892B1A
:1026900090FB81F98093830222C00E944E088091B2
:1026A000820287FB222720F991E0922790FB87F98D
:1026B00014C081E00E942E0F12C08091820284FB20
:1026C000222720F991E0922790FB84F906C080919F
:1026D0008202982F909590FB80F9809382028091DE
:1026E0008202909183020E94A80E0E944E0880E010
:1026F00001C081E0DF91CF910895CF93DF938631C0
:102700009C4541F5EB010E94A10D982F8A812091F3
:10271000040130910501882379F09A7A81E009F467
:1027200080E080935B02911102C069E201C065E321
:10273000C9010E9448150AC080915B02811102C044
:1027400069E201C065E3C9010E944A150E94E30DD8
:1027500080E001C081E0DF91CF9108950F931F9336
:10276000CF93DF93C42FD22FFC0182818823C9F03D
:1027700040935E020E94EE1590935D0280935C028E
:1027800080E28C0F883008F057C0C77081E001C02C
:10279000880FCA95EAF7DF91CF911F910F910C94A2
:1027A000BA0580915E02481330C080915C0290911E
:1027B0005D020E940616883C910538F510E21D0F57
:1027C000CD17B9F080E28C0F883040F4C77081E0FB
:1027D00001C0880FCA95EAF70E94C105183028F594
:1027E00081E09D2F977001C0880F9A95EAF70E94AB
:1027F000BA05802F0E94B1051830F0F4D77081E03F
:1028000001C0880FDA95EAF70AC080E28C0F8830A1
:1028100098F4C77081E001C0880FCA95EAF7DF918C
:10282000CF911F910F910C94C105802FDF91CF9113
:102830001F910F910C94B105DF91CF911F910F91D2
:1028400008950F939C01CB01243F4CE5340731F1EF
:1028500088F4293DFCE53F07D9F02A3D4CE53407D3
:1028600079F1283D3C45A9F506E221EE41EE68EDFF
:102870007CE52BC0263FFCE53F07E1F0A8F0273FB1
:102880003C4539F507E225EE46EE67EF7CE51DC0D5
:1028900007E225EE45EE69ED7CE517C006E221EE84
:1028A00040EE64EF7CE511C007E225EE44EE65EFF3
:1028B0007CE50BC006E221EE42EE66EF7CE505C04A
:1028C00008E221E045EE6AED7CE50E94AE1380E06F
:1028D00008C0FC018281882319F010925E0201C0B9
:1028E00081E00F91089580E090E008958FEF9FEFD1
:1028F00008950895862F0E94F51181E090E00895D3
:10290000EFE5F2E01382128288EE93E0A0E0B0E0FF
:1029100084839583A683B78389E791E0918380833D
:102920000895CF92DF92EF92FF920F931F93CF9370
:10293000DF936C01EB017B01E40EF51E00E010E07B
:10294000CE15DF0561F06991D601ED91FC91019002
:10295000F081E02DC6010995080F191FF1CFC801BC
:10296000DF91CF911F910F91FF90EF90DF90CF906B
:10297000089590938901809388010895909372023D
:10298000809371020895E0917102F0917202309784
:1029900021F00190F081E02D099480E00895E0910C
:1029A0007102F0917202309721F00280F381E02DE4
:1029B0000994089520916F02309170022817390709
:1029C00071F09093700280936F02E0917102F09128
:1029D0007202309721F00680F781E02D0994089566
:1029E00020916D0230916E022817390771F0909393
:1029F0006E0280936D02E0917102F0917202309745
:102A000021F00084F185E02D09940895FC013296AF
:102A100097E080E0915029F021912223D9F38F5F34
:102A2000F9CF0895662349F0FC013296089621916A
:102A3000621729F0E817F907D1F780E0089581E0DF
:102A400008959C01FC0132969FEF80E0419146176A
:102A500089F09F3F19F4411101C0982F8F5F863094
:102A6000A9F79F3F39F0F901E90FF11D97FDFA959C
:102A70006283089508959C012A5F3F4FFC014281C3
:102A8000461301C01282019682179307B9F7089581
:102A90000C9421150C943B15029626E0FC01119232
:102AA0002A95E9F7089508950C94531583E08093CF
:102AB00073020C945415811102C081E001C082E0C0
:102AC000809373020C9454150C945B1581E08093F1
:102AD00073020C9454150C94661508950C946D159E
:102AE0000C946E150C946D150C946D150C946D155D
:102AF000CF930E9474150E94D1010E947215C0E00C
:102B00008C2F0E941F02811104C0CF5FC031C1F71A
:102B100001C081E0CF91089508951F920F920FB6E2
:102B20000F9211248F939F93AF93BF938091740260
:102B3000811113C08091840290918502A091860238
:102B4000B09187024196A11DB11D8093840290939C
:102B50008502A0938602B0938702BF91AF919F91A7
:102B60008F910F900FBE0F901F90189580918C023F
:102B7000843031F10E942E041092740220E488E126
:102B800090E00FB6F894A895809360000FBE209354
:102B9000600083B7817F846083BF83B7816083BF18
:102BA0007894889583B78E7F83BF0FB6F894A895E5
:102BB00080916000886180936000109260000FBE79
:102BC00008950E944E080C94320482E084BD93E084
:102BD00095BD9AEF97BD80936E0008952FB7F89436
:102BE0008091840290918502A0918602B091870223
:102BF0002FBF08952FB7F8946091840270918502D9
:102C000080918602909187022FBF08959C014FB753
:102C1000F8948091840290918502A0918602B091EF
:102C200087024FBF821B930B089578941F920F92D7
:102C30000FB60F9211248F939F93AF93BF93809100
:102C4000840290918502A0918602B091870201963C
:102C5000A11DB11D8093840290938502A0938602EA
:102C6000B0938702BF91AF919F918F910F900FBE4C
:102C70000F901F90189587E797E79093010880932E
:102C800000089AE088E10FB6F894A8958093600058
:102C90000FBE90936000FFCF809180020895089549
:102CA000CF93DF9321E02093E9002FEF3091E800EC
:102CB000215035FD06C035ED3A95F1F700002111A0
:102CC000F5CF2091E80025FF14C0EC0140E050E072
:102CD00068E070E00E945C188091E8008E77809335
:102CE000E80088E0FE01A8E7B2E001900D928A9525
:102CF000E1F7DF91CF910895809375027093770289
:102D00006093760280918C02843001F582E080939A
:102D1000E9008FEF9091E800815095FD06C095ED98
:102D20009A95F1F700008111F5CF8091E80085FFB9
:102D30000DC040E050E063E070E085E792E00E9463
:102D40005C188091E8008E778093E8000895BC01BC
:102D500084E00C947C16BC0183E00C947C160895EE
:102D600080918B02811109C00E94ED190E944A1ABC
:102D70008091E20084608093E200089510928B02BB
:102D800008950C946B156091880281E0611101C077
:102D900080E00C94561590918C0281E0943009F0FB
:102DA00080E0609188020C945B1542E061EC81E068
:102DB0000E94661942E261EC82E00E9466199091DD
:102DC0008C0281E0943009F080E0609188020C94DC
:102DD000641580918E02833009F461C030F4813033
:102DE00071F0823009F49AC008958A3009F486C0DF
:102DF0008B3009F46CC0893009F0A8C020C08091E4
:102E00008D02813A09F0A2C08091E800877F80930B
:102E1000E8008091910290919202892B21F468E060
:102E200088E792E003C060E080E090E070E00E94FC
:102E3000A7188091E8008B778093E800089580912F
:102E40008D02813209F082C08091910290919202AC
:102E5000029708F07BC08091E800877F8093E800AC
:102E60008091E80082FD05C080918C028111F8CF2D
:102E70006DC02091F3008091F20090E0922B0297B8
:102E800031F48091F100813011F0863021F480918D
:102E9000F100809380028091E8008B7753C080918D
:102EA0008D02813A09F052C0809191029091920274
:102EB000892B09F04BC08091E800877F8093E80060
:102EC0008091E80080FFFCCF8091120136C0809194
:102ED0008D028132D9F58091910290919202892BD5
:102EE000A9F58091E800877F8093E8000E949B19F4
:102EF00080918F02809312010C944E0880918D0274
:102F0000813221F58091E800877F8093E8000E945C
:102F10009B198091900280938102089580918D0287
:102F2000813AA1F48091E800877F8093E800809146
:102F3000E80080FFFCCF809181028093F1008091B6
:102F4000E8008E778093E8000C949B19089584B76D
:102F5000877F84BF0FB6F894A89580916000886140
:102F600080936000109260000FBE90E080E80FB682
:102F7000F89480936100909361000FBE0C946615E5
:102F80000E94ED190E944A1AE2EEF0E0808184600E
:102F9000808378940C94DF1C86E091E00C94BE143E
:102FA00080918C028530A9F480918C02853079F46F
:102FB0000E94B61580918A028823B1F30E94781589
:102FC000882391F30E9446180E944E08EDCF0C947E
:102FD000E115089508950C94ED17292F3327233018
:102FE0003105C9F060F42130310581F0223031051E
:102FF00009F044C08BE390E026E132E043C0213287
:103000003105E1F02232310549F138C082E190E02A
:1030100021E532E037C099278130910549F028F049
:10302000029761F5E8EDF1E005C0E2E1F2E002C0EF
:10303000E8E0F2E0849190E09F0124C06115710501
:1030400041F061307105D1F489E090E021E432E093
:1030500019C089E090E028E232E014C061157105E2
:1030600041F06130710551F482E390E023E632E0F3
:1030700009C080E490E025E932E004C080E090E0FF
:1030800020E030E0FA0131832083089580E189BD9A
:1030900082E189BD09B400FEFDCF8091D8008F7D0B
:1030A0008093D8008091E00082608093E00080915E
:1030B000E00081FDFCCF0895CF92DF92EF92FF9266
:1030C0000F931F93CF93DF93EC018B017A010E9442
:1030D000BA19811133C0E114F10439F0F70180818C
:1030E0009181081B190BC80FD91FC12CD12C0115B8
:1030F000110519F18091E80085FD16C08091E80066
:103100008E778093E800E114F10449F0F7018081A3
:103110009181C80ED91ED182C08285E00FC00E9465
:10312000BA19882321F30AC089918093F1000150D4
:103130001109FFEFCF1ADF0ADACF80E0DF91CF91DC
:103140001F910F91FF90EF90DF90CF900895209105
:103150009302309194022617370748F061157105E4
:1031600039F42091E8002E772093E80001C0B901DE
:10317000FC0120E06115710579F180918C028823B2
:10318000F1F18530F1F18091E80083FD3CC0809140
:10319000E80082FD2EC08091E80080FFEBCF2091F7
:1031A000F3008091F20090E0922B6115710551F0CF
:1031B0008830910538F421912093F1006150710914
:1031C0000196F3CF21E0089709F020E08091E80014
:1031D0008E778093E800CECF2111CFCF0AC08091A7
:1031E0008C02882361F0853061F08091E80083FDD6
:1031F0000AC08091E80082FFF2CF80E0089582E06B
:10320000089583E0089581E008952091930230911C
:1032100094022617370748F06115710539F420919B
:10322000E8002E772093E80001C0B901FC0120E0FE
:103230006115710591F180918C02882309F440C0D9
:10324000853009F43FC08091E80083FD3DC0809146
:10325000E80082FD2FC08091E80080FFE9CF209137
:10326000F3008091F20090E0922B6115710559F006
:103270008830910540F424912093F10031966150FB
:1032800071090196F2CF21E0089709F020E08091C2
:10329000E8008E778093E800CBCF2111CCCF0AC015
:1032A00080918C02882361F0853061F08091E80084
:1032B00083FD0AC08091E80082FFF2CF80E008958C
:1032C00082E0089583E0089581E00895982F973073
:1032D00068F59093E900981739F07091EC0020910F
:1032E000ED005091F00003C0242F762F50E021FD17
:1032F00002C09F5FECCF3091EB003E7F3093EB003C
:103300003091ED003D7F3093ED003091EB00316066
:103310003093EB007093EC002093ED005093F0009D
:103320002091EE0027FDE5CF80E008958F70809317
:10333000E90081E0089580918D0287FF11C080919E
:10334000E80082FD05C080918C028111F8CF11C088
:103350008091E8008B770BC080918C02882349F024
:103360008091E80080FFF8CF8091E8008E7780930D
:10337000E80008952091E4003091E50095E6409141
:10338000EC00842F817040FF23C08091E80080FD15
:103390001DC080918C02882399F0853099F080912E
:1033A000EB0085FD11C04091E4005091E500241729
:1033B000350729F3915011F09A01E1CF84E0089587
:1033C00082E0089583E0089581E0089580E0089503
:1033D0004091E80042FFDDCF08950E945B1A0E94F1
:1033E000631AE0EEF0E0808181608083E8EDF0E038
:1033F00080818F77808319BCA7EDB0E08C918E7FA0
:103400008C9380818F7E808310928B0208950F931E
:103410001F93CF93DF930E945B1A0E94631AC8ED3B
:10342000D0E088818F7788838881806888838881CD
:103430008F7D888319BC10928C02109288021092A2
:103440008A021092890200EE10E0F80180818B7FE1
:10345000808388818160888342E060E080E00E9410
:103460006619E1EEF0E080818E7F8083E2EEF0E08D
:10347000808181608083808188608083F801808181
:103480008E7F8083888180618883DF91CF911F91B7
:103490000F910895E8EDF0E080818F7E8083E7ED65
:1034A000F0E080818160808384E082BF81E080934E
:1034B0008B020C94071AE8EDF0E080818E7F808308
:1034C0001092E20008951092DA001092E10008953F
:1034D0001F920F920FB60F9211242F933F934F9389
:1034E0005F936F937F938F939F93AF93BF93EF936C
:1034F000FF938091E10082FF0BC08091E20082FF88
:1035000007C08091E1008B7F8093E1000E94DE1C68
:103510008091DA0080FF1FC08091D80080FF1BC01F
:103520008091DA008E7F8093DA008091D90080FF4D
:103530000DC080E189BD82E189BD09B400FEFDCFE7
:1035400081E080938C020E94B01605C019BC1092D5
:103550008C020E94BE168091E10080FF19C080910C
:10356000E20080FF15C08091E2008E7F8093E20030
:103570008091E20080618093E2008091D8008062B7
:103580008093D80019BC85E080938C020E94C316FA
:103590008091E10084FF30C08091E20084FF2CC064
:1035A00080E189BD82E189BD09B400FEFDCF809133
:1035B000D8008F7D8093D8008091E1008F7E80932A
:1035C000E1008091E2008F7E8093E2008091E20032
:1035D00081608093E20080918802882311F084E06A
:1035E00007C08091E30087FD02C081E001C083E055
:1035F00080938C020E94CB168091E10083FF29C04A
:103600008091E20083FF25C08091E100877F809355
:10361000E10082E080938C02109288028091E100A8
:103620008E7F8093E1008091E2008E7F8093E200A4
:103630008091E20080618093E20042E060E080E0FF
:103640000E9466198091F00088608093F0000E94CB
:10365000C116FF91EF91BF91AF919F918F917F9193
:103660006F915F914F913F912F910F900FBE0F90EF
:103670001F9018951F920F920FB60F9211242F933F
:103680003F934F935F936F937F938F939F93AF93EA
:10369000BF93CF93DF93EF93FF93C091E900CF7077
:1036A0008091EC00D82FD17080FDD0E81092E90015
:1036B0008091F000877F8093F00078940E947E1BB9
:1036C0001092E9008091F00088608093F000CD2B8B
:1036D000CF70C093E900FF91EF91DF91CF91BF913F
:1036E000AF919F918F917F916F915F914F913F919A
:1036F0002F910F900FBE0F901F9018951F93CF938F
:10370000DF93CDB7DEB7AA970FB6F894DEBF0FBE32
:10371000CDBFEDE8F2E08091F100819322E0E53940
:10372000F207C9F70E94E9168091E80083FF2EC1D5
:1037300080918D0290918E02492F50E04A305105C0
:1037400008F024C1FA01EE59FF4F0C94FA1C80389E
:1037500021F0823809F01AC108C080918902909145
:103760008A02992389F082600FC0809191028F7044
:10377000873008F00BC18093E9008091EB0085FB56
:10378000882780F91092E9009091E800977F909344
:10379000E8008093F1001092F100D1C0282F2D7F16
:1037A00009F0F4C0882319F0823061F0EFC08091F5
:1037B0008F02813009F0EAC0933009F080E08093F5
:1037C0008A022EC080918F0281112AC080919102BD
:1037D0008F702FEF280F263008F0D8C08093E900B3
:1037E0002091EB0020FF1CC0933021F48091EB006E
:1037F000806214C09091EB0090619093EB0021E007
:1038000030E0A90102C0440F551F8A95E2F74093AA
:10381000EA001092EA008091EB0088608093EB0050
:103820001092E9008091E800877F8093E8000E9471
:103830009B19ACC08111AAC010918F021F77809193
:10384000E3008078812B8093E3008091E800877FFC
:103850008093E8000E949B198091E80080FFFCCFD4
:103860008091E30080688093E300111102C082E040
:1038700001C083E080938C0289C08058823008F0B8
:1038800085C080918F02909190028C3D53E0950706
:1038900079F583E08A838AE289834FB7F894DE0161
:1038A000139620E03EE051E2E32FF0E05093570002
:1038B000E49120FF03C0E295EF703F5FEF708E2F21
:1038C00090E0EA3010F0C79601C0C0968D939D93AA
:1038D0002F5F243149F74FBF8091E800877F8093A5
:1038E000E8006AE270E0CE0101960E94A71816C0B7
:1038F0006091910270919202AE014F5F5F4F0E9402
:10390000EB17BC01892B09F441C09091E800977F27
:103910009093E80089819A810E9405198091E800BE
:103920008B778093E80032C0803881F58091E80081
:10393000877F8093E800809188028093F1008091D6
:10394000E8008E7772CF811121C080918F02909113
:10395000900299270297D4F48091E800877F8093A2
:10396000E80080918F02809388020E949B198091C9
:103970008802811106C08091E30087FD02C081E0CA
:1039800001C084E080938C020E94D5168091E800EB
:1039900083FF0AC08091E800877F8093E8008091D0
:1039A000EB0080628093EB00AA960FB6F894DEBF1E
:1039B0000FBECDBFDF91CF911F9108950895CF9392
:1039C00080918C028823A1F0C091E900CF70909182
:1039D000EC00892F817090FD80E8C82B1092E900DF
:1039E0008091E80083FD0E947E1BCF70C093E900A8
:1039F000CF910895EE0FFF1F0590F491E02D0994EB
:103A0000FB01DC0104C08D910190801921F441502B
:103A10005040C8F7881B990B0895F999FECF92BDC5
:103A200081BDF89A992780B50895A8E1B0E042E0F9
:103A300050E00C94411D262FF999FECF92BD81BD17
:103A4000F89A019700B4021639F01FBA20BD0FB6DC
:103A5000F894FA9AF99A0FBE08950396272F0E94B8
:103A60001C1D0E941B1D252F0E941C1D242F0C9421
:103A70001C1D0196272F0E941C1D0C941B1DDC0190
:103A8000CB01FC01F999FECF06C0F2BDE1BDF89A69
:103A9000319600B40D9241505040B8F70895F89413
:023AA000FFCF56
:103AA200FFFFC80038024C165016AF16AB16A71609
:103AB2004F1601E200E900EA00B500B600B700CDFA
:103AC200008301CC008A0192019401210223022485
:103AD200022502260227022A02B300B4006F0070F8
:103AE20000818283E200E900EA00B500B600B70077
:103AF200CD008301CC008A019201940121022302AC
:103B020024022502260227022A02B300B4006F0013
:103B12007000818283000000007A1491147314767D
:083B22001476147914791400E3
:00000001FF
